:020000000141BC
:03000B00758CDC15
:10000E00DA307A19B2B7DB2A7B040560E560B45AA0
:10001E00217560500561E561B45617756150056232
:10002E00E562B45A0D7562500563E563B456037507
:10003E006350327590FF75B0F030B47A75504075DC
:10004E00517975522475533075541975551275566C
:10005E0002755778755800755910755A7F7560502E
:10006E007561507562507563507A197B0475A8825C
:10007E00758901758CDC758A00D28CD2B0A8608629
:10008E0090D9FE7590FFC2B0D2B1A8618690D9FE0C
:10009E007590FFC2B1D2B2A8628690D9FE7590FF5C
:1000AE00C2B2D2B3A863B85002785A8690D9FE7500
:1000BE0090FFC2B30189756712756608756547753D
:1000CE00647975B0007590FF7905D2B0856490DFC4
:1000DE00FE7590FFC2B0D2B1856590DFFE7590FFC0
:1000EE00C2B1D2B2856690DFFE7590FFC2B2D2B3B6
:1000FE00856790DFFE7590FFC2B3D8CED9CC74FF62
:10010E00F59075B00FC2E0C3F590D8FED9FCB2B72A
:10011E003370F47A10D8FED9FCDAFA7F08D3F59052
:10012E00D8FED9FCB2B733DFF47590FF53B0809090
:10013E00019875647F75657F75667F75677F74003E
:10014E0093B480028042856667856566856465F531
:10015E0064B2B7D2B0856490D8FE7590FFC2B0D2AB
:10016E00B1856590D8FE7590FFC2B1D2B28566900A
:10017E00D8FE7590FFC2B2D2B3856790D8FE759047
:10018E00FFC2B3D9CEA380B60141637977407F7F9A
:10019E007F7F120847087F797F7F7F7F4640210649
:1001AE007F03117F61062F24117F2F0807404624FD
:1001BE00117F7F7F7F2447402411477F24062B40E9
:1001CE002B7F2F0807404624117F7F7F7F3F3F24E0
:1001DE00023F79243F244040243F3F7F7F7F7F8032
:00000001FF
